:020000009C283A
:08000800FF00030E8301A000BC
:100010000A08A1008A010408A2000E280313831213
:10002000861B1828FA0A04307A0603192128192891
:10003000FA01061A3428FB0A04307B0603192B2820
:1000400035282830F400F201F501F60A3C30760636
:10005000031D3528F6012830F400F201F70A0C30B0
:1000600077060319F7013528FB010B1D92280B11A8
:10007000FF308100F40A32307406031D5728013026
:10008000F202031845280230F200F401F50A3C3070
:100090007506031D5728F501F60A3C307606031D48
:1000A0005728F601F70A0C3077060319F701F20812
:1000B000031D61280F3085007708F9007608F800E5
:1000C000922879087218780883169B001C147218FD
:1000D0007528F908031D6F2812309A0075280A3018
:1000E0001A0203187528F0309A048030F0000030AE
:1000F000F10019307402031882289A0E0030F000C3
:100100004030F1000F309A057008721871081A0417
:10011000831285004030740783169B001C141A0854
:10012000831295008B162208840021088A00200E75
:100130008300FF0E7F0E09008030F0004030F10098
:100140000230F200F401F501F601F701F801F901BE
:10015000FA01FB01FF30A400FF30A5003030D720AA
:100160009730D5208312031307309F00640081016C
:1001700083166F3081006400683081008312FF3085
:10018000810083168E15FF3092008312950197121D
:100190001712043092000F3097000B118B168B173B
:1001A000CF3085000000D228D428A500D928A4008B
:0E01B000DC2825086600080024086500080009
:02400E00703F01
:024200000000bc
:024202000100b9
:024204000200b6
:024206000300b3
:024208000400b0
:02420a000500ad
:02420c000600aa
:02420e000700a7
:024210000800a4
:024212000900a1
:02421400100098
:02421600110095
:02421800120092
:02421a0013008f
:02421c0014008c
:02421e00150089
:02422000160086
:02422200170083
:02422400180080
:0242260019007d
:02422800200074
:02422a00210071
:02422c0022006e
:02422e0023006b
:02423000240068
:02423200250065
:02423400260062
:0242360027005f
:0242380028005c
:02423a00290059
:02423c00300050
:02423e0031004d
:0242400032004a
:02424200330047
:02424400340044
:02424600350041
:0242480036003e
:02424a0037003b
:02424c00380038
:02424e00390035
:0242500040002c
:02425200410029
:02425400420026
:02425600430023
:02425800440020
:02425a0045001d
:02425c0046001a
:02425e00470017
:02426000480014
:02426200490011
:02426400500008
:02426600510005
:02426800520002
:02426a005300ff
:02426c005400fc
:02426e005500f9
:024270005600f6
:024272005700f3
:024274005800f0
:024276005900ed
:02428000f0004c
:02428200ec004e
:02428400e10057
:02428600cf0067
:02428800b8007c
:02428a009d0095
:02428c007f00b1
:02428e006100cd
:024290004400e8
:024292002b00ff
:02429400160012
:02429600000026
:02429800000024
:02429a00000022
:02429c0016000a
:02429e002b00f3
:0242a0004400d8
:0242a2006100b9
:0242a4007f0099
:0242a6009d0079
:0242a800b8005c
:0242aa00cf0043
:0242ac00e1002f
:0242ae00ec0022
:0242b000f0001c
:0242b200f0001a
:0242b400ec001c
:0242b600e10025
:0242b800cf0035
:0242ba00b8004a
:0242bc009d0063
:0242be007f007f
:0242c00061009b
:0242c2004400b6
:0242c4002b00cd
:0242c6001600e0
:0242c8000000f4
:0242ca000000f2
:0242cc000000f0
:0242ce001600d8
:0242d0002b00c1
:0242d2004400a6
:0242d400610087
:0242d6007f0067
:0242d8009d0047
:0242da00b8002a
:0242dc00cf0011
:0242de00e100fd
:0242e000ec00f0
:0242e200f000ea
:00000001FF
